:040000008A017628D3
:08000800F300F30E030EF400F7
:10001000040EF5000A0EF6008A110A12C129C92938
:100020008A150A12122A8A150A12182A8A150A1221
:10003000512B8A150A126F2B8A150A12342C8A1535
:100040000A12192D8A150A121F2E8A150A12B72EA6
:100050008A110A16D62C8A110A16602D8A110A16E0
:10006000A22D8A110A16122E8A110A16322F8A110F
:100070000A16712F8A110A16952F8A110A16A12FB6
:100080008A110A16AC2F8A110A16F52F8A150A163C
:100090000D288A150A165E288A150A16B8288A15A8
:1000A0000A16C9288A150A16DB288A150A167A291B
:1000B0008A150A16AD298A150A16F5298A150A160F
:1000C000392A8A150A16992A8A150A16BD2A8A1506
:1000D0000A16A92B8A150A16B12B8A150A168A2C1C
:1000E0008A150A16352D8A150A16592D07308316DA
:1000F00003139F00C030FB00A830FC00FD0102305C
:10010000FE00C030810034208A110A125330831659
:100110000313E1003A208A110A1274308316031384
:10012000E1003A208A110A12613083160313E100BC
:100130003A208A110A12723083160313E1003A2022
:100140008A110A12743083160313E1003A208A11CF
:100150000A12693083160313E1003A208A110A1249
:100160006E3083160313E1003A208A110A126730B9
:1001700083160313E1003A208A110A1220308316F5
:100180000313E1003A208A110A1275308316031313
:10019000E1003A208A110A12703083160313E1003D
:1001A0003A208A110A122E3083160313E1003A20F6
:1001B0008A110A122E3083160313E1003A208A11A5
:1001C0000A122E3083160313E1003A208A110A1214
:1001D00010208A110A1283120313DF013130DC0070
:1001E000E201E3015030E40013208A110A12831265
:1001F0000313DB00E60116208A110A12831603138B
:10020000E6010130E70043208A110A1243308316C9
:100210000313E1003A208A110A126F308316031388
:10022000E1003A208A110A126D3083160313E100AF
:100230003A208A110A12703083160313E1003A2023
:100240008A110A126C3083160313E1003A208A11D6
:100250000A12653083160313E1003A208A110A124C
:10026000743083160313E1003A208A110A126530B4
:1002700083160313E1003A208A110A122E308316E6
:100280000313E1003A208A110A120130831203138A
:10029000DA0073208A110A1237208A110A12831693
:1002A0000313C30125208A110A128312DB00DB0825
:1002B0000319B8298316D9014730DA004530DB002D
:1002C0005430DC002030DD002B208A110A1283120A
:1002D000DB00DB08031985290F208A110A1283121B
:1002E0000313E70119208A110A1283120313E20192
:1002F000E3015030E40013208A110A128312031321
:10030000DB00E60116208A110A1283160313C301CB
:1003100025208A110A128312DB0037208A110A1263
:1003200083160313E601E70143208A110A128312A0
:100330000313DE0110305E020318B3298316D501C2
:1003400028208A110A128312DD008316E1003A2068
:100350008A110A12F001831203135E08013E03188A
:10036000F00ADE009A298316E0012E208A110A1273
:10037000013083120313DA0073208A110A124F2905
:10038000C029760E8A00750E8400740E8300730EE9
:10039000090037208A110A12533083160313E10033
:1003A0003A208A110A12653083160313E1003A20BD
:1003B0008A110A126E3083160313E1003A208A1163
:1003C0000A12643083160313E1003A208A110A12DC
:1003D000693083160313E1003A208A110A126E3045
:1003E00083160313E1003A208A110A12673083163C
:1003F0000313E1003A208A110A12203083160313F6
:10040000E1003A208A110A12683083160313E100D2
:100410003A208A110A12743083160313E1003A203D
:100420008A110A126D3083160313E1003A208A11F3
:100430000A126C3083160313E1003A208A110A1263
:100440002E3083160313E1003A208A110A122E304F
:1004500083160313E1003A208A110A122E30831604
:100460000313E1003A208A110A12013083120313A8
:10047000DA0073208A110A12EC011C208A110A1278
:1004800083120313EE014830EF001F208A110A1275
:1004900083120313EE015430EF001F208A110A1259
:1004A00083120313EE015430EF001F208A110A1249
:1004B00083120313EE015030EF001F208A110A123D
:1004C00083120313EE012F30EF001F208A110A124E
:1004D00083120313EE013130EF001F208A110A123C
:1004E00083120313EE012E30EF001F208A110A122F
:1004F00083120313EE013030EF001F208A110A121D
:1005000083120313EE012030EF001F208A110A121C
:1005100083120313EE013230EF001F208A110A12FA
:1005200083120313EE013030EF001F208A110A12EC
:1005300083120313EE013030EF001F208A110A12DC
:1005400083120313EE012030EF001F208A110A12DC
:1005500083120313EE014F30EF001F208A110A129D
:1005600083120313EE014B30EF001F208A110A1291
:1005700083120313EE010D30EF001F208A110A12BF
:1005800083120313EE010A30EF001F208A110A12B2
:1005900083120313EE014330EF001F208A110A1269
:1005A00083120313EE016F30EF001F208A110A122D
:1005B00083120313EE016E30EF001F208A110A121E
:1005C00083120313EE017430EF001F208A110A1208
:1005D00083120313EE016530EF001F208A110A1207
:1005E00083120313EE016E30EF001F208A110A12EE
:1005F00083120313EE017430EF001F208A110A12D8
:1006000083120313EE012D30EF001F208A110A120E
:1006100083120313EE017430EF001F208A110A12B7
:1006200083120313EE017930EF001F208A110A12A2
:1006300083120313EE017030EF001F208A110A129B
:1006400083120313EE016530EF001F208A110A1296
:1006500083120313EE013A30EF001F208A110A12B1
:1006600083120313EE012030EF001F208A110A12BB
:1006700083120313EE017430EF001F208A110A1257
:1006800083120313EE016530EF001F208A110A1256
:1006900083120313EE017830EF001F208A110A1233
:1006A00083120313EE017430EF001F208A110A1227
:1006B00083120313EE012F30EF001F208A110A125C
:1006C00083120313EE016830EF001F208A110A1213
:1006D00083120313EE017430EF001F208A110A12F7
:1006E00083120313EE016D30EF001F208A110A12EE
:1006F00083120313EE016C30EF001F208A110A12DF
:1007000083120313EE010D30EF001F208A110A122D
:1007100083120313EE010A30EF001F208A110A1220
:1007200083120313EE010D30EF001F208A110A120D
:1007300083120313EE010A30EF001F208A110A1200
:1007400083120313EE013C30EF001F208A110A12BE
:1007500083120313EE016830EF001F208A110A1282
:1007600083120313EE017430EF001F208A110A1266
:1007700083120313EE016D30EF001F208A110A125D
:1007800083120313EE016C30EF001F208A110A124E
:1007900083120313EE013E30EF001F208A110A126C
:1007A00083120313EE012030EF001F208A110A127A
:1007B00083120313EE010D30EF001F208A110A127D
:1007C00083120313EE010A30EF001F208A110A1270
:1007D00083120313EE013C30EF001F208A110A122E
:1007E00083120313EE016830EF001F208A110A12F2
:1007F00083120313EE016530EF001F208A110A12E5
:1008000083120313EE016130EF001F208A110A12D8
:1008100083120313EE016430EF001F208A110A12C5
:1008200083120313EE013E30EF001F208A110A12DB
:1008300083120313EE010D30EF001F208A110A12FC
:1008400083120313EE010A30EF001F208A110A12EF
:1008500083120313EE013C30EF001F208A110A12AD
:1008600083120313EE017430EF001F208A110A1265
:1008700083120313EE016930EF001F208A110A1260
:1008800083120313EE017430EF001F208A110A1245
:1008900083120313EE016C30EF001F208A110A123D
:1008A00083120313EE016530EF001F208A110A1234
:1008B00083120313EE013E30EF001F208A110A124B
:1008C00083120313EE015430EF001F208A110A1225
:1008D00083120313EE014330EF001F208A110A1226
:1008E00083120313EE015030EF001F208A110A1209
:1008F00083120313EE015F30EF001F208A110A12EA
:1009000083120313EE014930EF001F208A110A12EF
:1009100083120313EE015030EF001F208A110A12D8
:1009200083120313EE012030EF001F208A110A12F8
:1009300083120313EE014330EF001F208A110A12C5
:1009400083120313EE016F30EF001F208A110A1289
:1009500083120313EE016D30EF001F208A110A127B
:1009600083120313EE017030EF001F208A110A1268
:1009700083120313EE012030EF001F208A110A12A8
:1009800083120313EE015730EF001F208A110A1261
:1009900083120313EE016530EF001F208A110A1243
:1009A00083120313EE016230EF001F208A110A1236
:1009B00083120313EE012030EF001F208A110A1268
:1009C00083120313EE017030EF001F208A110A1208
:1009D00083120313EE016130EF001F208A110A1207
:1009E00083120313EE016730EF001F208A110A12F1
:1009F00083120313EE016530EF001F208A110A12E3
:100A000083120313EE013C30EF001F208A110A12FB
:100A100083120313EE012F30EF001F208A110A12F8
:100A200083120313EE017430EF001F208A110A12A3
:100A300083120313EE016930EF001F208A110A129E
:100A400083120313EE017430EF001F208A110A1283
:100A500083120313EE016C30EF001F208A110A127B
:100A600083120313EE016530EF001F208A110A1272
:100A700083120313EE013E30EF001F208A110A1289
:100A800083120313EE010D30EF001F208A110A12AA
:100A900083120313EE010A30EF001F208A110A129D
:100AA00083120313EE013C30EF001F208A110A125B
:100AB00083120313EE012F30EF001F208A110A1258
:100AC00083120313EE016830EF001F208A110A120F
:100AD00083120313EE016530EF001F208A110A1202
:100AE00083120313EE016130EF001F208A110A12F6
:100AF00083120313EE016430EF001F208A110A12E3
:100B000083120313EE013E30EF001F208A110A12F8
:100B100083120313EE010D30EF001F208A110A1219
:100B200083120313EE010A30EF001F208A110A120C
:100B300083120313EE013C30EF001F208A110A12CA
:100B400083120313EE016230EF001F208A110A1294
:100B500083120313EE016F30EF001F208A110A1277
:100B600083120313EE016430EF001F208A110A1272
:100B700083120313EE017930EF001F208A110A124D
:100B800083120313EE012030EF001F208A110A1296
:100B900083120313EE016230EF001F208A110A1244
:100BA00083120313EE016730EF001F208A110A122F
:100BB00083120313EE016330EF001F208A110A1223
:100BC00083120313EE016F30EF001F208A110A1207
:100BD00083120313EE016C30EF001F208A110A12FA
:100BE00083120313EE016F30EF001F208A110A12E7
:100BF00083120313EE017230EF001F208A110A12D4
:100C000083120313EE013D30EF001F208A110A12F8
:100C100083120313EE013030EF001F208A110A12F5
:100C200083120313EE013030EF001F208A110A12E5
:100C300083120313EE013030EF001F208A110A12D5
:100C400083120313EE013030EF001F208A110A12C5
:100C500083120313EE016630EF001F208A110A127F
:100C600083120313EE016630EF001F208A110A126F
:100C700083120313EE012030EF001F208A110A12A5
:100C800083120313EE017430EF001F208A110A1241
:100C900083120313EE016530EF001F208A110A1240
:100CA00083120313EE017830EF001F208A110A121D
:100CB00083120313EE017430EF001F208A110A1211
:100CC00083120313EE013D30EF001F208A110A1238
:100CD00083120313EE016630EF001F208A110A12FF
:100CE00083120313EE016630EF001F208A110A12EF
:100CF00083120313EE016630EF001F208A110A12DF
:100D000083120313EE016630EF001F208A110A12CE
:100D100083120313EE013030EF001F208A110A12F4
:100D200083120313EE013030EF001F208A110A12E4
:100D300083120313EE013E30EF001F208A110A12C6
:100D400083120313EE010D30EF001F208A110A12E7
:100D500083120313EE010A30EF001F208A110A12DA
:100D600083120313EE013C30EF001F208A110A1298
:100D700083120313EE016830EF001F208A110A125C
:100D800083120313EE013130EF001F208A110A1283
:100D900083120313EE013E30EF001F208A110A1266
:100DA00083120313EE014830EF001F208A110A124C
:100DB00083120313EE016530EF001F208A110A121F
:100DC00083120313EE016C30EF001F208A110A1208
:100DD00083120313EE016C30EF001F208A110A12F8
:100DE00083120313EE016F30EF001F208A110A12E5
:100DF00083120313EE012030EF001F208A110A1224
:100E000083120313EE015730EF001F208A110A12DC
:100E100083120313EE016F30EF001F208A110A12B4
:100E200083120313EE017230EF001F208A110A12A1
:100E300083120313EE016C30EF001F208A110A1297
:100E400083120313EE016430EF001F208A110A128F
:100E500083120313EE013C30EF001F208A110A12A7
:100E600083120313EE012F30EF001F208A110A12A4
:100E700083120313EE016830EF001F208A110A125B
:100E800083120313EE013130EF001F208A110A1282
:100E900083120313EE013E30EF001F208A110A1265
:100EA00083120313EE010D30EF001F208A110A1286
:100EB00083120313EE010A30EF001F208A110A1279
:100EC00083120313EE013C30EF001F208A110A1237
:100ED00083120313EE017030EF001F208A110A12F3
:100EE00083120313EE013E30EF001F208A110A1215
:100EF00083120313EE014830EF001F208A110A12FB
:100F000083120313EE016F30EF001F208A110A12C3
:100F100083120313EE017730EF001F208A110A12AB
:100F200083120313EE012030EF001F208A110A12F2
:100F300083120313EE016130EF001F208A110A12A1
:100F400083120313EE017230EF001F208A110A1280
:100F500083120313EE016530EF001F208A110A127D
:100F600083120313EE012030EF001F208A110A12B2
:100F700083120313EE017930EF001F208A110A1249
:100F800083120313EE016F30EF001F208A110A1243
:100F900083120313EE017530EF001F208A110A122D
:100FA00083120313EE012030EF001F208A110A1272
:100FB00083120313EE017430EF001F208A110A120E
:100FC00083120313EE016F30EF001F208A110A1203
:100FD00083120313EE016430EF001F208A110A12FE
:100FE00083120313EE016130EF001F208A110A12F1
:100FF00083120313EE017930EF001F208A110A12C9
:101000008A150A1283120313EE013F308A150A1261
:10101000EF008A110A121F208A150A128312031385
:10102000EE013C30EF008A110A121F208A150A12C5
:1010300083120313EE012F30EF008A110A121F20D2
:101040008A150A1283120313EE017030EF008A1121
:101050000A121F208A150A1283120313EE013E3072
:10106000EF008A110A121F208A150A12F00131308E
:10107000831203135F070318F00ADC00F0015F0816
:10108000013E0318F00ADF00093C031CDF01831254
:101090000313EE013C30EF008A110A121F208A155B
:1010A0000A1283120313EE017030EF008A110A1244
:1010B0001F208A150A1283120313EE013E30EF003F
:1010C0008A110A121F208A150A1283120313EE01D5
:1010D0005030EF008A110A121F208A150A1283125B
:1010E0000313EE016130EF008A110A121F208A15E6
:1010F0000A1283120313EE016730EF008A110A12FD
:101100001F208A150A1283120313EE016530EF00C7
:101110008A110A121F208A150A1283120313EE0184
:101120002030EF008A110A121F208A150A1283123A
:101130000313EE017230EF008A110A121F208A1584
:101140000A1283120313EE016530EF008A110A12AE
:101150001F208A150A1283120313EE017130EF006B
:101160008A110A121F208A150A1283120313EE0134
:101170007530EF008A110A121F208A150A12831295
:101180000313EE016530EF008A110A121F208A1541
:101190000A1283120313EE017330EF008A110A1250
:1011A0001F208A150A1283120313EE017430EF0018
:1011B0008A110A121F208A150A1283120313EE01E4
:1011C0003A30EF008A110A121F208A150A12831280
:1011D0000313EE012030EF008A110A121F208A1536
:1011E0000A1283120313EE015C08EF008A110A123F
:1011F0001F208A150A1283120313EE013C30EF0000
:101200008A110A121F208A150A1283120313EE0193
:101210002F30EF008A110A121F208A150A1283123A
:101220000313EE017030EF008A110A121F208A1595
:101230000A1283120313EE013E30EF008A110A12E4
:101240001F208A150A1283120313EE012030EF00CB
:101250008A110A121F208A150A1283120313EE0143
:101260000D30EF008A110A121F208A150A1283120C
:101270000313EE010A30EF008A110A121F208A15AB
:101280000A1283120313EE013C30EF008A110A1296
:101290001F208A150A1283120313EE012F30EF006C
:1012A0008A110A121F208A150A1283120313EE01F3
:1012B0006230EF008A110A121F208A150A12831267
:1012C0000313EE016F30EF008A110A121F208A15F6
:1012D0000A1283120313EE016430EF008A110A121E
:1012E0001F208A150A1283120313EE017930EF00D2
:1012F0008A110A121F208A150A1283120313EE01A3
:101300003E30EF008A110A121F208A150A1283123A
:101310000313EE012030EF008A110A121F208A15F4
:101320000A1283120313EE010D30EF008A110A1224
:101330001F208A150A1283120313EE010A30EF00F0
:101340008A110A121F208A150A1283120313EE0152
:101350003C30EF008A110A121F208A150A128312EC
:101360000313EE012F30EF008A110A121F208A1595
:101370000A1283120313EE016830EF008A110A1279
:101380001F208A150A1283120313EE017430EF0036
:101390008A110A121F208A150A1283120313EE0102
:1013A0006D30EF008A110A121F208A150A1283126B
:1013B0000313EE016C30EF008A110A121F208A1508
:1013C0000A1283120313EE013E30EF008A110A1253
:1013D0001F208A150A1283120313EE012030EF003A
:1013E0008A110A121F208A150A1283120313EE01B2
:1013F0000D30EF008A110A121F208A150A1283127B
:101400000313EE010A30EF008A110A121F208A1519
:101410000A1283160313C2018A110A1222208A15A6
:101420000A1208008A110A1231208A150A120800CD
:10143000F0010930F200831203136208F100083052
:101440000310F00CF10C0318F007F20B212A7108BD
:10145000E5000E30E0006208043C0318302A003436
:1014600003179201F0010930F2001830F100031364
:1014700062080310F00CF10C0318F007F20B3A2A83
:101480007108A03EF1000318F00A7108013EF10056
:101490000318F00A710803179300013094008A11B1
:1014A0000A1255208A150A12831203179201F001BD
:1014B0000930F2001830F100031362080310F00C39
:1014C000F10C0318F007F20B5F2A7108A03EF1003F
:1014D0000318F00A71080E3EF1000318F00A7108B3
:1014E0000317930003136308031794008A110A1269
:1014F00055208A150A12831203179201F001093050
:10150000F2001830F100031362080310F00CF10C24
:101510000318F007F20B862A7108A03EF1000318A9
:10152000F00A71080E3EF1000318F00A7108013E3E
:10153000F1000318F00A71080317930003136408FD
:10154000031794008A110A1255208A150A12F00115
:10155000831203136208203E840070088313800006
:10156000831203179201F00103136208003E03186F
:10157000F00A03179300023094008A110A125520D2
:101580008A150A12831203136208203E8400831313
:101590000008003C031DD22A8A110A126A208A150B
:1015A0000A12C22A831203136208203E84008313A6
:1015B00000080239003C031DDE2A003483120313A5
:1015C000620803179E008A110A1264208A150A1203
:1015D000F001F101831203136508003E0318F10ABC
:1015E000A03E8400700883138000F001F101831293
:1015F00003136508013E0318F10AA03E8400700839
:1016000083138000F001F101831203136508023E89
:101610000318F10AA03E8400700883138000F001D3
:10162000F101831203136508033E0318F10AA03E7B
:101630008400700883138000F001F101831203130A
:101640006508043E0318F10AA03E84007008831365
:101650008000F001F101831203136508053E0318B1
:10166000F10AA03E8400700883138000F001F101AC
:10167000831203136508063E0318F10AA03E840096
:10168000700883138000F001F101831203136508D1
:10169000073E0318F10AA03E8400700883138000FF
:1016A00001340E3083120313E000F0016608203E7F
:1016B0008400700883138000831203179201F001E5
:1016C00003136608003E0318F00A0317930008305E
:1016D00094008A110A1255208A150A1208000E3049
:1016E00083120313E000EA016430EB00EA08031DF3
:1016F000152CF0010930F2000330F10067080310E7
:10170000F00CF10C0318F007F20B802B7108E03E8F
:10171000F1000318F00A7108023EF1000318F00A04
:10172000710803179C00F0010930F2000C30F10041
:10173000031367080310F00CF10C0318F007F20B09
:101740009B2B7108103EF1000318F00A7108083E47
:10175000F1000318F00A710803179D008A110A129C
:1017600061208A150A12770883120313E8007808AB
:10177000E900F0010930F2000330F10067080310BE
:10178000F00CF10C0318F007F20BC02B7108E03ECF
:10179000F1000318F00A7108103EF1000318F00A76
:1017A000710803179C00F0010930F2000C30F100C1
:1017B000031367080310F00CF10C0318F007F20B89
:1017C000DB2B7108403EF1000318F00A7108031783
:1017D0009D008A110A1261208A150A127708831265
:1017E000031368020130031D0301FF390319012CA3
:1017F000780869020130031D0301FF390319012C28
:101800000130003C0319072C0130EA00762B01302F
:10181000D8008A110A1270208A150A12EB03EB080D
:10182000031D142C0130EA00762B83120313EB08FE
:101830000319332CF0016708203E840070088313DD
:101840008000831203179201F00103136708003E22
:101850000318F00A03179300103094008A110A123B
:1018600055208A150A120800F0010930F20083128F
:1018700003136C08F10004300310F00CF10C031892
:10188000F007F20B3D2C7108E1000E30E000031769
:101890009501F0010930F2001830F10003136C08D3
:1018A0000310F00CF10C0318F007F20B512C710827
:1018B000A03EF1000318F00A7108031796008A1180
:1018C0000A1258208A150A120313ED000E3C031861
:1018D000A42CF0010930F2000330F1006C08031071
:1018E000F00CF10C0318F007F20B702C7108E03EBD
:1018F000F1000318F00A7108113EF1000318F00A14
:10190000710803179C00F0010930F2000C30F1005F
:1019100003136C080310F00CF10C0318F007F20B22
:101920008B2C7108403EF1000318F00A7108043E48
:10193000F1000318F00A710803179D008A110A12BA
:1019400061208A150A12E02CF0010930F200033000
:10195000F100831203136C080310F00CF10C031850
:10196000F007F20BAD2C7108E03EF1000318F00A0D
:101970007108023EF1000318F00A710803179C0079
:10198000F0010930F2000C30F10003136C08031071
:10199000F00CF10C0318F007F20BC82C7108103E84
:1019A000F1000318F00A7108083EF1000318F00A6C
:1019B000710803179D008A110A1261208A150A1204
:1019C0007708F000F101831203136108003E031849
:1019D000F10A243E84007008831380007808F00028
:1019E000F101831203136108013E0318F10A243E3A
:1019F00084007008831380007908F000F1018312DD
:101A000003136108023E0318F10A243E84007008A3
:101A1000831380007A08F000F10183120313610838
:101A2000033E0318F10A243E8400700883138000EB
:101A30000800F0010930F200831203136E08F10070
:101A400004300310F00CF10C0318F007F20B222DF8
:101A50007108E1000E30E000F0016108003E03185B
:101A6000F00A243E84008313000883160313C00089
:101A7000F0010930F20083126E08F1000830031003
:101A8000F00CF10C0318F007F20B402D7108403EEA
:101A9000F1000318F00A7108F100F2016108013E3B
:101AA0000318F20A243E84008313000807397107E3
:101AB000F1000318F00A710883160313C1008A119C
:101AC0000A124C208A150A120E30EA008A110A12F4
:101AD00049208A150A124108EA008A110A1249208F
:101AE0008A150A124008EA008A110A1249208A154A
:101AF0000A1283126F088316EA008A110A1249201B
:101B00008A110A124F208A150A12F001F10183127C
:101B10006108003E0318F10A243E84008313000884
:101B2000013E0318F00AF000F1018312031361086B
:101B3000003E0318F10A243E8400700883138000DD
:101B4000F001831203136108003E0318F00A243EDB
:101B5000840083130008003C031D1E2EF001F101D8
:101B6000831203136108013E0318F10A243E840026
:101B700083130008013E0318F00AF000F1018312FC
:101B800003136108013E0318F10A243E8400700823
:101B900083138000F001831203136108013E0318D0
:101BA000F00A243E840083130008003C031D1E2E0F
:101BB000F001F101831203136108023E0318F10AD8
:101BC000243E840083130008013E0318F00AF0004D
:101BD000F101831203136108023E0318F10A243E47
:101BE0008400700883138000F001831203136108DE
:101BF000023E0318F00A243E840083130008003CD0
:101C0000031D1E2EF001F101831203136108033E30
:101C10000318F10A243E840083130008013E0318D0
:101C2000F00AF000F101831203136108033E031868
:101C3000F10A243E840070088313800008000E30EF
:101C400083120313E000F0010930F200831642080A
:101C5000F10004300310F00CF10C0318F007F20B44
:101C60002B2E71088312E100F0016108003E031879
:101C7000F00A243E840083130008F700F001831269
:101C800003136108013E0318F00A243E8400831305
:101C90000008F800F001831203136108023E0318E4
:101CA000F00A243E840083130008F900F001831237
:101CB00003136108033E0318F00A243E84008313D3
:101CC0000008FA00831203179801F0010930F200AE
:101CD0000C30F1008316031342080310F00CF10CD2
:101CE0000318F007F20B6E2E7108403EF100031846
:101CF000F00A71088312031799008A110A125B20F7
:101D00008A150A120230FF008A110A1267208A150A
:101D10000A12F001831603134208203E8400700863
:101D200083138000831203179201F00183160313BB
:101D30004208003E0318F00A831203179300203074
:101D400094008A110A1255208A150A128316031369
:101D50004208203E8400831300082039031DB62E5C
:101D60008A110A126A208A150A12A62E0800831602
:101D70000313C601C7010130C800CB01D001F00137
:101D80000930F2004308F10004300310F00CF10CAC
:101D90000318F007F20BC62E71088312E100F00160
:101DA0000930F20083164308F10008300310F00CEC
:101DB000F10C0318F007F20BD72E7108CF000E308C
:101DC0008312E000F00183164308203E840070086F
:101DD00083138000831603134308203E840083137B
:101DE00000084039031D0C2F831203179201F001E4
:101DF000831603134308003E0318F00A83120317E7
:101E00009300403094008A110A1255208A110A1258
:101E10006A208A150A12EA2EF0010930F200033016
:101E2000F1008316031343080310F00CF10C0318A0
:101E3000F007F20B152F7108E03EF1000318F00ACD
:101E40007108831203179C00F0010930F2000C3076
:101E5000F1008316031343080310F00CF10C031870
:101E6000F007F20B2D2F7108103EF1000318F00A55
:101E70007108831203179D008A110A1261208A15C6
:101E80000A12770883120313D4007808D500790862
:101E9000D6007A08D700F0010930F2000330F100D3
:101EA000831643080310F00CF10C0318F007F20B33
:101EB000532F7108E03EF1000318F00A7108013E4B
:101EC000F1000318F00A7108831203179C00F00157
:101ED0000930F2000C30F10083160313430803109D
:101EE000F00CF10C0318F007F20B702F7108103E84
:101EF000F1000318F00A7108043EF1000318F00A1B
:101F00007108831203179D008A110A1261208A1535
:101F10000A127708F000F101831203136108003EF2
:101F20000318F10A343E8400700883138000780897
:101F3000F000F101831203136108013E0318F10A56
:101F4000343E84007008831380007908F000F101AA
:101F5000831203136108023E0318F10A343E840021
:101F60007008831380007A08F000F10183120313D4
:101F70006108033E0318F10A343E8400700883139D
:101F80008000831203135408F000F1016108003E41
:101F90000318F10A343E84008313000870028A118A
:101FA0000A16031D11288A150A12831203135508F5
:101FB000F000F1016108013E0318F10A343E84008B
:101FC0008313000870028A110A16031D11288A154E
:101FD0000A12831203135608F000F1016108023E51
:101FE0000318F10A343E84008313000870028A113A
:101FF0000A16031D11288A150A12831203135708A3
:102000008A110A16F000F1016108033E0318F10A73
:10201000343E8400831300087002831603130319EF
:10202000C8018312031795018A110A16F0010930BD
:10203000F2001830F1008316031343080310F00C6C
:10204000F10C0318F007F20B1F287108A03EF100F5
:102050000318F00A71088312031796008A110A12F6
:1020600058208A110A1683160313C900F00070085D
:102070000F3C031D3C2845287008113C031D4128D6
:1020800045287008123C031D4B280830CD00C601BE
:102090000830CA0065287008103C031D5728063018
:1020A00083160313CD000230C600CA0165287008EC
:1020B000133C031D6328033083160313CD00C600B1
:1020C0000430CA0065280130D000C8080319D22C9A
:1020D000D0080319A32883125408F000F101610805
:1020E000003E0318F10A443E840070088313800008
:1020F000831203135508F000F1016108013E031833
:10210000F10A443E84007008831380008312031395
:102110005608F000F1016108023E0318F10A443E3E
:102120008400700883138000831203135708F000A3
:10213000F1016108033E0318F10A443E840070086F
:1021400083138000D22CF001831203136108003E38
:102150000318F00A343E8400831300088316031327
:10216000D100F00183126108013E0318F00A343EE9
:1021700084008313000883160313D200F001831236
:102180006108003E0318F00A343E840083130008FF
:10219000F000F101831203136108003E0318F10AF5
:1021A000443E8400700883138000F00183120313FF
:1021B0006108013E0318F00A343E840083130008CE
:1021C000F000F101831203136108013E0318F10AC4
:1021D000443E8400700883138000F00183120313CF
:1021E0006108023E0318F00A343E8400831300089D
:1021F000F000F101831203136108023E0318F10A93
:10220000443E8400700883138000F001831203139E
:102210006108033E0318F00A343E8400831300086B
:10222000F000F101831203136108033E0318F10A61
:10223000443E8400700883138000F001831203136E
:102240006108003E0318F00A343E8400831300083E
:1022500083160313C400F0010930F2004308F100B3
:1022600008300310F00CF10C0318F007F20B3229C0
:102270007108603EF1000318F00A7108F100F201E4
:1022800083126108013E0318F20A343E840083136E
:10229000000807397107F1000318F00A7108831666
:1022A0000313C5008A110A124C208A110A160E3037
:1022B000EA008A110A1249208A110A164508EA0022
:1022C0008A110A1249208A110A164408EA008A1162
:1022D0000A1249208A110A124F208A110A124C2030
:1022E0008A110A160F30EA008A110A1249208A114F
:1022F0000A16CB0101304D024B020318A129EF0150
:102300008A110A1252208A110A16F000F10183166E
:1023100003134F084B070318F10AA03E840070080E
:102320008313800083160313430883120317A4004A
:102330008A110A126D208A110A1683160313CB0A1A
:102340007A290130EF008A110A1252208A110A16E6
:10235000F000F101831603134F084B070318F10A2D
:10236000A03E84007008831380008A110A124F2057
:102370008A110A16430883120317A4008A110A124D
:102380006D208A110A16F001831603134F08003ED0
:102390000318F00AA03E8400831300080A3C0318C7
:1023A000B62AF001831603134308203E8400700808
:1023B00083138000831203179201F0018316031325
:1023C0004308003E0318F00A8312031793001030ED
:1023D00094008A110A1255208A110A1683160313D3
:1023E000C9080319172A831203179501F001093050
:1023F000F2001830F1008316031343080310F00CA9
:10240000F10C0318F007F20BFF297108A03EF10050
:102410000318F00A71088312031796008A110A1232
:1024200058208A110A1683160313C900EE29F701F2
:10243000F801F901FA01831203179801F00109303C
:10244000F2000C30F1008316031343080310F00C64
:10245000F10C0318F007F20B272A7108103EF10067
:102460000318F00A7108043EF1000318F00A71081D
:102470008312031799008A110A125B208A110A1627
:102480000230FF008A110A1267208A110A1683128D
:1024900003179801F0010930F2000C30F1008316A7
:1024A000031343080310F00CF10C0318F007F20BB0
:1024B000532A7108103EF1000318F00A71088312C4
:1024C000031799008A110A125B208A110A1602303A
:1024D000FF008A110A1267208A110A16F00183167A
:1024E00003134308203E8400700883138000831286
:1024F00003179201F001831603134308003E0318EB
:10250000F00A831203179300023094008A110A1212
:1025100055208A110A1683160313C908031DB42A0D
:10252000831203179501F0010930F2001830F10011
:102530008316031343080310F00CF10C0318F00783
:10254000F20B9C2A7108A03EF1000318F00A7108F2
:102550008312031796008A110A1258208A110A164C
:1025600083160313C9008B2AC801D22CF0018316ED
:1025700003134608F100F2014F08013E0318F20A66
:10258000A03E84008313000871070318F00A831625
:102590000313C600F0014F08013E0318F00AA03EE5
:1025A000840083130008831603134602031CC70A22
:1025B000F001831603134F08003E0318F00AA03EF3
:1025C00084008313000883160313C700F0014F082B
:1025D000003E0318F00AA03E84008313000883160F
:1025E0000313D300F0014F08013E0318F00AA03E88
:1025F00084008313000883160313D400F0014F08EE
:10260000013E0318F00AA03E8400831300088316DD
:102610000313CC00F0014F08013E0318F00AA03E5E
:10262000840083130008831603134A02F000700924
:10263000013EF000F1014F08013E0318F10AA03EEF
:102640008400700883138000F001831603134F0881
:10265000013E0318F00AA03E84008313000883168D
:1026600003134C0203184E2BF0014F08003E0318D1
:10267000F00AA03E840083130008013CF0007009BA
:10268000013EF000F101831603134F08003E0318CA
:10269000F10AA03E840070088313800083160313A0
:1026A0004608003C0318EF2BC603F001F10183122A
:1026B0006108003E0318F10A443E840083130008B9
:1026C000013E0318F00AF000F101831203136108C0
:1026D000003E0318F10A443E840070088313800012
:1026E000F001831203136108003E0318F00A443E10
:1026F000840083130008003C031D4E2BF001F10100
:10270000831203136108013E0318F10A443E84005A
:1027100083130008013E0318F00AF000F101831250
:1027200003136108013E0318F10A443E8400700857
:1027300083138000F001831203136108013E031824
:10274000F00A443E840083130008003C031DEE2B76
:10275000F001F101831203136108023E0318F10A2C
:10276000443E840083130008013E0318F00AF00081
:10277000F101831203136108023E0318F10A443E7B
:102780008400700883138000F00183120313610832
:10279000023E0318F00A443E840083130008003C04
:1027A000031DEE2BF001F101831203136108033EB8
:1027B0000318F10A443E840083130008013E031805
:1027C000F00AF000F101831203136108033E0318BD
:1027D000F10A443E84007008831380004E2B831658
:1027E00003134708003C0318662CC703F001F101EE
:1027F00083126108013E0318F10A443E84008313EA
:102800000008013E0318F00AF000F10183120313DF
:102810006108013E0318F10A443E840070088313E6
:102820008000F001831203136108013E0318F00ACF
:10283000443E840083130008003C031DEF2BF0018D
:10284000F101831203136108023E0318F10A443EAA
:10285000840083130008013E0318F00AF000F10120
:10286000831203136108023E0318F10A443E8400F8
:10287000700883138000F001831203136108023E85
:102880000318F00A443E840083130008003C031D33
:10289000652CF001F101831203136108033E031854
:1028A000F10A443E840083130008013E0318F00A35
:1028B000F000F101831203136108033E0318F10ACB
:1028C000443E8400700883138000EF2B83160313AB
:1028D000CE0183125708F000F1016108013E031890
:1028E000F10A443E8400831300087002031CAC2CE0
:1028F000831203135608F000F1016108023E031829
:10290000F10A443E8400831300087002031CAC2CBF
:10291000831203135508F000F1016108013E03180A
:10292000F10A443E8400831300087002031CAC2C9F
:10293000831203135408F000F1016108003E0318EC
:10294000F10A443E8400831300087002031CAC2C7F
:10295000013083160313CE0083160313C801013020
:102960004E02031DD22CF0014F08003E0318F00A5E
:10297000A03E840083130008003C0318C42CFF30E1
:1029800083160313C800D22CF001831603134F08DB
:10299000013E0318F00AA03E84008313000883164A
:1029A0000313C8008316031348080800F001093018
:1029B000F200831603135508F10004300310F00CE5
:1029C000F10C0318F007F20BDF2C71088312E10001
:1029D0000E30E000F0016108003E0318F00A343EBA
:1029E00084008313000883160313D700F001093015
:1029F000F2005508F10008300310F00CF10C031838
:102A0000F007F20BFD2C7108603EF1000318F00A8C
:102A10007108F100F20183126108013E0318F20A05
:102A2000343E84008313000807397107F10003184E
:102A3000F00A710883160313D8008A110A124C2079
:102A40008A110A160E30EA008A110A1249208A11E8
:102A50000A165808EA008A110A1249208A110A1631
:102A60005708EA008A110A1249208A110A124F20D7
:102A70008A110A124C208A110A160F30EA008A11B4
:102A80000A1249208A110A160130EF008A110A122F
:102A900052208A110A1683160313D6008A110A12CD
:102AA0004F208A110A16550883120317A4008A11B1
:102AB0000A126D208A110A1683160313560808009D
:102AC000013083160313DE000E308312E0008316FC
:102AD0005908D5008A110A1228208A110A16DF0027
:102AE0005A020319762D83160313DE015908D50007
:102AF0008A110A1228208A110A16DF005B020319C4
:102B0000842D83160313DE015908D5008A110A1299
:102B100028208A110A16DF005C020319922D831601
:102B20000313DE015908D5008A110A1228208A11E0
:102B30000A16DF005D020319A02D83160313DE01C0
:102B40005E0808000E3083120313E000F001093024
:102B5000F20083166008F10004300310F00CF10C51
:102B60000318F007F20BAE2D71088312E100F0019B
:102B70006108003E0318F00A443E840083130008F5
:102B8000F700F001831203136108013E0318F00AF5
:102B9000443E840083130008F800F00183120313FD
:102BA0006108023E0318F00A443E840083130008C3
:102BB000F900F001831203136108033E0318F00AC1
:102BC000443E840083130008FA008312031798011F
:102BD000F0010930F2000C30F10083160313600895
:102BE0000310F00CF10C0318F007F20BF12D710833
:102BF000103EF1000318F00A7108043EF1000318BA
:102C0000F00A71088312031799008A110A125B20D7
:102C10008A110A160230FF008A110A1267208A11EF
:102C20000A1608000E3083120313E00083160716FD
:102C30008715071431309300940194179101831282
:102C40009401941514169416031792019301803081
:102C500094008A110A1255208A110A16831203174A
:102C6000920180309300C03094008A110A125520DE
:102C70008A110A1683120317920181309300A8303B
:102C800094008A110A1255208A110A16831203171A
:102C900092018230930094018A110A1255208A1100
:102CA0000A16831203179201833093000A309400AE
:102CB0008A110A1255208A110A16831203179201EB
:102CC00084309300FF3094008A110A1255208A1133
:102CD0000A1683120317920185309300FF30940087
:102CE0008A110A1255208A110A16831203179201BB
:102CF00086309300FF3094008A110A1255208A1101
:102D00000A168312031792018730930094018A11E7
:102D10000A1255208A110A1683120317920188306D
:102D2000930094018A110A1255208A110A168312FF
:102D30000317920189309300083094008A110A1217
:102D400055208A110A168312031792018A309300C4
:102D5000DC3094008A110A1255208A110A16831257
:102D6000031792018B30930094018A110A125520A7
:102D70008A110A168312031792018C309300940172
:102D80008A110A1255208A110A168312031792011A
:102D90008D30930094018A110A1255208A110A1667
:102DA0008312031792018E3093007B0894008A11DE
:102DB0000A1255208A110A168312031792018F30C6
:102DC00093007C0894008A110A1255208A110A1671
:102DD000831203179201903093007D0894008A11AA
:102DE0000A1255208A110A16831203179201913094
:102DF00093007E0894008A110A1255208A110A163F
:102E000083120317920195309300553094008A1174
:102E10000A1255208A110A1683120317920196305E
:102E20009300553094008A110A1255208A110A160F
:102E300083120313A0010317920193010130940040
:102E40008A110A1255208A110A16831203132008C8
:102E50000139031D312F8A110A126A208A110A16BC
:102E6000252F08008316831603130608C039860031
:102E7000831202308312D8008A110A1270208A113C
:102E80000A1633308316E2008A110A123D208A1195
:102E90000A16323083160313E2008A110A123D200B
:102EA0008A110A162C3083160313E2008A110A12C3
:102EB0003D208A110A16063083160313E2008A1198
:102EC0000A123D208A110A160C3083160313E20001
:102ED0008A110A123D208A110A1237208A110A1615
:102EE0000800013083160313E2008A110A123D2004
:102EF0008A110A16013083120313D8008A110A12AC
:102F000070208A110A1602308316E2008A110A1212
:102F10003D208A110A16013083120313D8008A114A
:102F20000A1270208A110A1608008316031361081A
:102F3000E3001030E4008A110A1240208A110A16B8
:102F40000800831603136208E300E4018A110A12E1
:102F500040208A110A160800831603136308F00044
:102F6000F00CF00CF00C700C0F390F396404E50014
:102F700083120608C03983166504E50083128600B3
:102F80000130D8008A110A1270208A110A1686169A
:102F90000130D8008A110A1270208A110A1686128E
:102FA000831663080F396404E50083120608C039EC
:102FB00083166504E500831286000130D8008A116B
:102FC0000A1270208A110A1686160130D8008A115A
:102FD0000A1270208A110A1686120130D8008A114E
:102FE0000A1270208A110A16080083160313E708D4
:102FF000031DFD2F8030E700FF2FC030E700F001F8
:103000008A150A16670866070318F00AE2008A1193
:103010000A123D208A150A16080083160313E901D7
:103020006808F0007008003C8A150A16031D1D2868
:10303000013083160313E9005C287008013C031D6E
:103040002628023083160313E9005C287008023C2E
:10305000031D2F28043083160313E9005C28700831
:10306000033C031D3828083083160313E9005C284D
:103070007008043C031D4128103083160313E90037
:103080005C287008053C031D4A2820308316031372
:10309000E9005C287008063C031D53284030831665
:1030A0000313E9005C287008073C031D5C2880308E
:1030B00083160313E9005C286908080002308316B0
:1030C0000313E8008A110A1246208A150A16EB003B
:1030D00014086B05003C03196E2868280430E800CA
:1030E0008A110A1246208A150A16EC000330E800FD
:1030F0008A110A1246208A150A166C04EC00023066
:10310000E8008A110A1246208A150A166C04EC009F
:103110000130E8008A110A1246208A150A166C044A
:10312000EC00E8018A110A1246208A150A166C047E
:10313000EC0011086C05003C03199F289928E80150
:103140008A110A1246208A150A16EC0014086C052A
:10315000003C0319AC28A6286A0883129300831642
:10316000031314086B05003C0319B728AF280800A7
:1031700083160313E8018A110A1246208A150A16DB
:10318000ED00910411086D056D02031DC828C228C9
:103190000800023083160313E8008A110A12462041
:1031A0008A150A16EE00910411086E056E02031DC1
:1031B000DA28D428080083120317900102308316FE
:1031C0000313E8008A110A1246208A150A16831290
:1031D00003179100831603131408831203171105B4
:1031E000003C0319F428EA28043083160313E8008E
:1031F0008A110A1246208A150A16831203179100B3
:10320000033083160313E8008A110A1246208A1538
:103210000A16831203171104910002308316031358
:10322000E8008A110A1246208A150A16831203172B
:1032300011049100013083160313E8008A110A1269
:1032400046208A150A16831203171104910083166B
:103250000313E8018A110A1246208A150A168312FE
:103260000317110491008316031311088312031727
:103270001105003C03193D2933290330831603133C
:10328000E8008A110A1246208A150A1683120317CB
:1032900091008316031391048316031311088312FC
:1032A000031711051102031D56294C298316031318
:1032B000EF08031D5D2991125E2991160430E80084
:1032C0008A110A1246208A150A16831203179100E2
:1032D0008316031391048316031311088312031733
:1032E00011051102031D75296B2903131308031718
:1032F000900008008A110A124C208A150A168312BF
:1033000060088316EA008A110A1249208A150A16F3
:1033100083120317120883160313EA008A110A1294
:1033200049208A150A1683120317130883160313FC
:10333000EA008A110A1249208A150A168312031715
:10334000140883160313EA008A110A1249208A110D
:103350000A124F208A150A1608008A110A124C20F8
:103360008A150A16831260088316EA008A110A1267
:1033700049208A150A1683120317150883160313AA
:10338000EA008A110A1249208A150A1683120317C5
:10339000160883160313EA008A110A1249208A11BB
:1033A0000A124F208A110A124C208A150A16F001BF
:1033B00083126008013E0318F00A8316EA008A119E
:1033C0000A1249208A150A160130EF008A110A12E2
:1033D00052208A150A1697008A110A124F208A1560
:1033E0000A1683120317170808008A110A124C20C4
:1033F0008A150A16831260088316EA008A110A12D7
:1034000049208A150A168312031718088316031316
:10341000EA008A110A1249208A150A168312031734
:10342000190883160313EA008A110A1249208A1523
:103430000A167A08EA008A110A1249208A150A1621
:103440007908EA008A110A1249208A150A167808B2
:10345000EA008A110A1249208A150A167708EA003A
:103460008A110A1249208A110A124F208A150A1657
:1034700008008A110A124C208A150A168312600865
:103480008316EA008A110A1249208A150A16831245
:1034900003171A0883160313EA008A110A12492037
:1034A0008A150A16831203171B0883160313EA00F2
:1034B0008A110A1249208A110A124F208A110A120F
:1034C0004C208A150A16F00183126008013E031889
:1034D000F00A8316EA008A110A1249208A150A1690
:1034E000EF018A110A1252208A150A16FA00831671
:1034F0000313EF018A110A1252208A150A16F900E5
:1035000083160313EF018A110A1252208A150A1634
:10351000F800013083160313EF008A110A125220BB
:103520008A150A16F7008A110A124F208A150A1600
:10353000080001308312031795001C0896008A11B9
:103540000A1258208A150A160230FF008A110A1240
:1035500067208A150A16831203179A011D089B001B
:103560008A110A125E208A150A160230FF008A119B
:103570000A1267208A150A160800F701F801F901F6
:10358000FA01831203179801F0010930F2000C30A0
:10359000F1001E080310F00CF10C0318F007F20BF9
:1035A000CB2A7108103EF1000318F00A7108043E9E
:1035B000F1000318F00A710899008A110A125B20C1
:1035C0008A150A160230FF008A110A1267208A152E
:1035D0000A16831203179801F0010930F2000C302B
:1035E000F1001E080310F00CF10C0318F007F20BA9
:1035F000F32A7108103EF1000318F00A71089900CF
:103600008A110A125B208A150A160230FF008A11FD
:103610000A1267208A150A16831203179501F00112
:103620000930F2001830F1001E080310F00CF10C04
:103630000318F007F20B162B7108A03EF1000318D7
:10364000F00A710896008A110A1258208A150A1683
:103650009F000E3C031C352B1230FA003430F90069
:1036600003130108F8000109F700831203179801FA
:10367000F0010930F2000C30F1001E080310F00CCC
:10368000F10C0318F007F20B3F2B7108403EF100DC
:103690000318F00A710899008A110A125B208A1532
:1036A0000A160230FF008A110A1267208A150A16CC
:1036B000831203179801F0010930F2000C30F10079
:1036C0001E080310F00CF10C0318F007F20B622B2C
:1036D0007108403EF1000318F00A7108043EF10041
:1036E0000318F00A710899008A110A125B208A15E2
:1036F0000A160230FF008A110A1267208A150A167C
:10370000831203179801F0010930F2000C30F10028
:103710001E080310F00CF10C0318F007F20B8A2BB3
:103720007108103EF1000318F00A7108083EF1001C
:103730000318F00A710899008A110A125B208A1591
:103740000A160230FF008A110A1267208A150A162B
:1037500008000230FF0200000000FF0BAB2B00004E
:10376000080083120317A0010E300313E0000708BE
:103770000317A1000139003C031D862C9501083078
:1037800096008A110A1258208A150A16A200A00073
:10379000220803197C2C221CE52B9501043096008D
:1037A0008A110A1258208A150A16A30092010830BD
:1037B0009300013094008A110A1255208A150A16C6
:1037C0008312031723080313A00083120317A21CFC
:1037D000012C9501053096008A110A1258208A158D
:1037E0000A16A300920108309300023094008A1157
:1037F0000A1255208A150A16831203172308031389
:10380000A10083120317221D1D2C9501063096007E
:103810008A110A1258208A150A16A300920108304C
:103820009300043094008A110A1255208A150A1652
:103830008312031723080313A20083120317A21D88
:10384000382C9501073096008A110A1258208A15E3
:103850000A16A30092010830930094008A110A12FC
:1038600055208A150A168312031723080313A30091
:1038700083120317221E462C920108309300103049
:1038800094008A110A1255208A150A16831203170A
:10389000A21E542C920108309300203094008A110B
:1038A0000A1255208A150A1683120317221F622C4A
:1038B000920108309300403094008A110A1255207A
:1038C0008A150A1683120317A21F702C9201083062
:1038D0009300803094008A110A1255208A150A1626
:1038E000831203179501083096008A110A12582096
:1038F0008A150A16A200C82B920108309300FF30E7
:1039000094008A110A1255208A150A168312031789
:1039100020080800F0010930F20083120317240880
:10392000F10004300310F00CF10C0318F007F20B57
:10393000932C71080313E100F001F1016108003ECE
:103940000318F10A343E840083130008013E031873
:10395000F00AF000F101831203136108003E03181E
:10396000F10A343E8400700883138000F001831252
:1039700003136108003E0318F00A343E84008313E9
:103980000008003C031D342DF001F10183120313E4
:103990006108013E0318F10A343E840083130008D5
:1039A000013E0318F00AF000F101831203136108CD
:1039B000013E0318F10A343E84007008831380002E
:1039C000F001831203136108013E0318F00A343E2C
:1039D000840083130008003C031D342DF001F10125
:1039E000831203136108023E0318F10A343E840077
:1039F00083130008013E0318F00AF000F10183125E
:103A000003136108023E0318F10A343E8400700873
:103A100083138000F001831203136108023E031830
:103A2000F00A343E840083130008003C031D342D4B
:103A3000F001F101831203136108033E0318F10A38
:103A4000343E840083130008013E0318F00AF0009E
:103A5000F101831203136108033E0318F10A343E97
:103A600084007008831380000800B93083120313A8
:103A7000D90000000000000000000000000000006D
:103A80000000000000000000000000000000000036
:103A90000000000000000000000000000000000026
:103AA00000000000D90B3A2D0000D80B352D000086
:103AB0000800FA3083120313D8008A110A1270200A
:103AC0008A150A16FA30D8008A110A1270208A154F
:103AD0000A16FA30D8008A110A1270208A150A16BE
:103AE000FA30D8008A110A1270208A150A16DA0BE9
:043AF000592D080044
:00000001FF
